:105CD90001130000090101240200000301FA040074
:105CE900FA0500030A0A5A0B001E0C00FA0D0003FC
:105CF9000E00030F0164100096120132130AFA1400
:105D0900010215000217010A1801FA1905321A01D0
:105D19000A1B01FA1C05321FFFFF20FFFF23011E8A
:105D29002400642A00FA2B00FA2C50782D003D2E0D
:105D390000462F001E3000643250783432FA3501A3
:105D490064360164370150380A643C00643E003C03
:105D59003F000140FFFF411450420A5A430AC84418
:105D690005324500B44600FA4701484802034C0091
:105D7900FA4EFFFF500404510596520A32530B465E
:105D8900540A96560102570546580002590A465ABE
:105D990032FA5B010A5C0A325E000A5F00FE61FFAB
:105DA900FF6402116600026701016A0A3C6B000088
:105DB9006C32967300007400007801327901327EEA
:105DC900FFFF81FFFF84FFFF8500AF860001870089
:105DD900FA89010A8A00009900009D0A969E00012D
:105DE9009FFFFFFAFAFA00000901012402000003EB
:105DF90001FA0400FA0500030A0A5A0B001E0C00F6
:105E0900FA0D00030E00030F01641000961201320F
:105E1900130AFA14010215000017010A1801FA19E8
:105E290005321A010A1B01FA1C05321FFFFF20FF68
:105E3900FF23011E2400642A00FA2B00FA2C507853
:105E49002D003D2E00462F001E300064325078345C
:105E590032FA350164360164370150380A643C006E
:105E6900643E003C3F000140FFFF411450420A5A82
:105E7900430AC84405324500B44600FA470124489C
:105E890002024C00FA4EFFFF500404510596520AD3
:105E990032530B46540A96560101570546580001DC
:105EA900590A465A32FA5B010A5C0A325E000A5FF5
:105EB90000FE61FFFF6402116600026701016A0AC0
:105EC9003C6B00006C32967300007400007801325C
:105ED9007901327EFFFF81FFFF84FFFF85FFFF8687
:105EE900FFFF87FFFF8901028A00009900009D0AD0
:105EF900969E00019FFFFFFAFAFA0065006F00798C
:105F09000083008D009700A100AC00B600C000CA54
:105F190000D400DE00E800F2005B0063006A007252
:105F2900007A008200890091009900A100A800B0C0
:105F390000B800BF00C700CF00D600DF00E600EEC2
:105F490000F600400046004C00520059005F006511
:105F5900006B00710077007D00830089008F009538
:105F6900009C00A200A800AE00B400BA00C000C6A0
:0E5F790000CC00D200D900DF00E500EB00F103
:1035E700900049E0D3940440149007BAE0FEA3E0AA
:1035F700FF905CDB1260C0E493F59980129007BAE4
:10360700E0FEA3E0FF905DEF1260C0E493F59990B0
:1036170007BAE0FEA3E0FF905CD9E493FC74019342
:10362700FDEFB50507EEB50403754D009007BA1217
:1036370060A72285F97285FA737E017F00E5731210
:103647006099E5722FFF50010E8E598F5A90001323
:10365700E0FCA3E0FDEF2DFDEE3CFC8C5B8D5C22D6
:1036670075A71085F97285FA737E017F00E57312DD
:103677006099E5722FFF50010E8E598F5A9000DC2A
:10368700E0B40210AC2CAD2DEF2DFDEE3CFC8C5BB5
:103697008D5C8016AE59AF5A900013E0FCA3E0FD95
:1036A700EF2DFDEE3CFC8C5B8D5C22AE59AF5A745E
:1036B7000A8E048F05FF1260898C5B8D5CAE59AF53
:1036C7005A740A8E048F05FF1260B48C598D5AE51F
:1036D7005A45596013740AC3955AFFE49559FE8EEB
:1036E700598F5A785B1260EDE572A85BB80015D365
:1036F700955C4010E572C3955CFFE4955BFE8E5BBD
:103707008F5C8010E5722424C3955CFFE4955BFE13
:103717008E5B8F5CAE5BAF5C74246F4E700B755C19
:1037270023755B0075720180037572002290008A11
:10373700E0B40104C2108002D21090008BE0B40103
:1037470004C2118002D2119000C8E075F0DCA4FF1A
:10375700AEF0740A8E048F05FF1260899007B0ECF3
:10376700F0A3EDF0A20D401674038C068D071260CE
:103777009974011200399007AEEEF0A3EFF07E01C5
:103787007F00900086E01260999000C9E08E048F58
:1037970005FF126089740AFF1260898D5F9000D25D
:1037A700E075F0DCA4FFAEF0740A8E048F05FF12FB
:1037B70060899007B4ECF0A3EDF09000D4E06013BB
:1037C7009000D4E0F5F0741684FF7E00EF9007BEFA
:1037D700F0800674649007BEF09000CAE090006E17
:1037E700F0900114E0900058F09000A3E090005A88
:1037F700F09000CCE090005BF0900078E090005CE7
:10380700F09000FEE0900061F074E390006DF0909E
:1038170000B3E0B40B0874E390006DF0805A900099
:10382700B3E0B419129000C9E0905EEE12008CE488
:103837009390006DF080419000B3E0B41E129000A9
:10384700C9E0905F0C12008CE49390006DF0802823
:103857009000B3E0B428129000C9E0905F361200E0
:103867008CE49390006DF0800F9000B3E0B44608AD
:103877009000AAE090006DF0900071E0FE9000B01B
:10388700E0B50633900073E0FE9000CEE0B5062762
:10389700900072E0FE9000DCE0B5061B900075E03A
:1038A700FE900083E0B5060F900074E0FE9000BE26
:1038B700E06E70030239FE900049E0C3940550089A
:1038C70074029000FFF080149000DCE06008740838
:1038D7009000FFF08006740A9000FFF0900083E0EC
:1038E700B4010674009000E9F0900083E0B402068A
:1038F70074009000CEF0900083E0B403067400904B
:1039070000DBF09000CEE0D39401401474189001CE
:1039170001F074009006C8F074009006C9F0800C9E
:103927007400900101F074189006C8F09000B0E0A0
:103937006014741A900097F074009006D0F0740029
:103947009006D1F0800C7400900097F0741A9006DE
:10395700D0F09000B0E0B402147419900098F0749D
:10396700009006CCF074009006CDF0800C740090A7
:103977000098F074199006CCF09000DCE0700E749B
:10398700059006DCF074069006E0F080187400904D
:1039970006DCF074009006DDF074009006E0F07429
:1039A700009006E1F0D2269000B0E0900071F09010
:1039B70000DCE0900072F09000CEE0900073F09091
:1039C70000BEE0900074F0900083E0900075F090E6
:1039D7000083E0900059F09000BEE090005DF09009
:1039E70000DCE090005EF09000B0E090005FF090A7
:1039F70000CEE0900060F09000E6E0B40117900080
:103A07001F740FF0A374FFF0900021E4F0A3F0748B
:103A1700029000E6F09000E6E0B40341900021E058
:103A2700FEA3E0FF90001FE0FCA3E0FD1260E57439
:103A3700101260997408120039EF90006AF0EF7065
:103A47000674FF90006AF074009000E6F090002082
:103A5700E090006BF090001FE090006CF090007712
:103A6700E090003BF090003BE0241290003CF09087
:103A7700003CE0D39424400B90003CE0C394249096
:103A8700003CF090003FE4F090003BE0B4240C9041
:103A9700003F7401F090003B7401F0900040E4F0A7
:103AA70090003CE0B4240C9000407401F090003C7E
:103AB7007401F0900077E0FE9000DAE02E9000426B
:103AC700F0900042E064126007900042E0B42406E0
:103AD700900042E004F0900042E0D39424400B9021
:103AE7000042E0C39424900042F0900042E0D39457
:103AF70012400D900042E0C39412900043F0800AF8
:103B0700900042E02412900043F07550129000BDDF
:103B1700E090003DF090003DE075F01284AFF07E3C
:103B270000EF4E700690003DE004F090003DE0B4D9
:103B3700490690003D7401F090003DE0D394244085
:103B47000F90003DE0C3942490003DF0D220800206
:103B5700C22090003DE0D39412400D90003DE0C399
:103B6700941290003EF0800A90003DE024129000ED
:103B77003EF022C293C294C291C292C287C290E51C
:103B8700B554EFF5B5E5B554DFF5B5C296C295C2A4
:103B9700A0C297C2A2C2A1E5B554BFF5B5E5B55419
:103BA7007FF5B5E5B554FBF5B5C212755D469000D6
:103BB700C0E07005756C028003756C037554007561
:103BC700530090000874FFF0A374DCF0C217C21909
:103BD70074C8900033F074C8900037F075520075C0
:103BE7005100C20D754600E56EB40903756E007588
:103BF7006200900015E4F0A3F0756F10C215C216AD
:103C07009007B0E0FEA3E0FF7403126099740112FD
:103C170000399007AEEEF0A3EFF0C20275560075BB
:103C2700550090000CE4F0A3F0C2277558007557B3
:103C370000900082E075F032A4FDACF090001DEC1E
:103C4700F0A3EDF0C2372285F97285FA737E017F02
:103C570000E573126099E5722FFF50010E8E598FA0
:103C67005AAC5BAD5CEF2DFDEE3CFC8C5B8D5CD202
:103C770093D294E55CF5FBE55BF5FCE55CF5E9E5DE
:103C87005BF5EA9000BEE0B40314D291D292E55CF2
:103C9700F5EBE55BF5ECE55CF5EDE55BF5EE22753F
:103CA700A71085F97285FA737E017F00E5731260AC
:103CB70099E5722FFF50010E8E598F5A7E017F763C
:103CC7009000FBE0126099AC59AD5AED2FFFEC3E26
:103CD700FE8E5B8F5CE55CF5FDE55BF5FE90006EA7
:103CE700E4F075A7007412900045F02285F97285FB
:103CF700FA737E017F00E573126099E5722FFF501A
:103D0700010E8E598F5A9007B0E0FCA3E0FDEF2D0E
:103D1700FDEE3CFC8C5B8D5CE55CF5FDE55BF5FE43
:103D2700220563229000BEE0B403539000DCE0B4A8
:103D3700012EA2D8B34004C293C287A2D9B34004CC
:103D4700C294C290A2DAB34008C291E5B554EFF528
:103D5700B5A2DBB34008C292E5B554DFF5B5801CC8
:103D6700A2D8B34002C293A2D9B34002C294A2DA46
:103D7700B34002C291A2DBB34002C292801EA2D816
:103D8700B3400AC2939000DCE06002C287A2D9B3B5
:103D9700400AC2949000DCE06002C290A2DCB3400B
:103DA70004C296C29575D8402285A77175A710A23F
:103DB700D8B34002C287A2D9B34002C290A2DAB3F5
:103DC7004006E5B554EFF5B5A2DBB34006E5B554BB
:103DD700DFF5B5A2DCB340089000CAE090006EF0B2
:103DE70075D8408571A722900047E4936406600266
:103DF70080FE74C89007B6F8E4F0E8A3F075B50044
:103E070075840175A70075FFA0900041E4F075C99E
:103E17001075A70F75A1C775A70075D90075CE0CCA
:103E270075A70F75F1FE75F2FF75F30775F47875D1
:103E3700A4BA75A5FF75A60775AE0075AFFF75D453
:103E47008175D5FF75D6FF75D7FF75A70075A201D8
:103E570075A14775F80975D80075D90475DA09751C
:103E6700DB0975DC0975DD0975DE0975D84075A7AD
:103E77001075D80075D90475DA0975DB0975DC0981
:103E870075DD0975DE0975D84075A70075E60875F3
:103E9700E71075BC0175BE0475BD6C75BE0775BDB1
:103EA700A075BE0875BD0175BC0075BB1875BC2033
:103EB70075BA0875E88075D11375A70F75E1057593
:103EC700E20075C740123B7A759700759780740AB0
:103ED7001260797597C0E5975420700280F8758F46
:103EE7000275A700D2AF75980075A90C75A70F7555
:103EF700AB4375ADFB75AC1E75A71075C91875CAB0
:103F07000075CB0075C80475A700758912758E04F6
:103F1700758C00758A00C2A9D28C758D00758B00CF
:103F2700D2ABD28E75EF0675D944C29974C8F5091C
:103F37007508001200E375B5001204E37463900777
:103F4700B6F8E4F0E8A3F012036F74C89007B6F868
:103F5700E4F0E8A3F07464F5097508001200E39033
:103F67000059E0900083F0C21D900083E0D39403D2
:103F770040067400900083F0900083E09058F1F8B9
:103F87002828738028A2B44002D21D802075A70F6D
:103F970075F30F75A700A2A34002D21D800F75A766
:0D3FA7000F75F31775A700A2A44002D21DEC
:0C58F100023F8A023F8C023F94023FA558
:103FB400A21DB34066757208E572D3940E5020E5D5
:103FC400729007B6F8E4F0E8A3F012023E7464F5C8
:103FD400097508001200E37872740126F650D9744A
:103FE400029000BFF0900083E0D394034006740075
:103FF400900083F0900083E09058FDF828287380A7
:104004001674009000E9F0800E74009000CEF080E9
:074014000674009000DBF0D0
:0C58FD0002400302400502400D0240156D
:10401B00D21C8064757201E572D394075020E5724F
:10402B009007B6F8E4F0E8A3F012023E7464F509C9
:10403B007508001200E37872740126F650D97401EA
:10404B009000BFF0900083E0D3940340067400907F
:10405B000083F0900083E0905909F82828738016AC
:10406B0074009000E9F0800E74009000CEF0800692
:06407B0074009000DBF070
:0C59090002406902406B02407302407BC8
:10408100C21C900058E0900114F0900059E090009B
:1040910083F090005AE09000A3F090005BE0900064
:1040A100CCF090005CE0900078F090005DE0900032
:1040B100BEF090005EE09000DCF090005FE09000C8
:1040C100B0F0900060E09000CEF0900061E09000D0
:1040D100FEF09000C9E07006740A9000C9F09000EB
:1040E100AAE0700674E39000AAF09000B0E004909A
:1040F1000071F0123734E5B54401F5B5740690004E
:1041010047F07401900048F0740390004AF0740580
:1041110090004BF0740E90004CF0740590004DF03F
:10412100900049E0B40406740490004DF0740090CE
:10413100004EF07400900053F07400900054F0743D
:1041410001900055F07400900056F074FF900057F4
:10415100F0743390014DF0743690014EF0742D904F
:10416100014FF07431900150F07420900151F074BE
:1041710034900152F07443900153F07479900154DA
:10418100F0746C900155F07420900156F0742090F9
:104191000157F07420900158F07420900159F07487
:1041A1002090015AF0742090015BF09000E5E090BE
:1041B100006AF090009CE090006BF090009DE09010
:1041C100006CF0A2B6B3920EA2B3B3920FA2A4B345
:1041D1009223A2B4B39224A2A3B39225900066E4E1
:1041E100F0756E00743A900776F074FD900777F0E1
:1041F100900067E4F09007B0E0FEA3E0FF740312C3
:10420100609974011200399007AEEEF0A3EFF075DA
:104211006D01900045E4F0C222756200C213D21410
:10422100C202757000C229D203C22AD204C22BD2A3
:1042310005C22CD206C22DD207C22ED208C22FD25D
:1042410009C230D20AC231D20BC232D20CC21EC252
:104251001FC220C221C22612009E755E00756A002F
:104261007560007564327565007566007567007567
:104271006800756900900015E4F0A3F0756B00D239
:10428100B2D2A4D2B0D2B1D2A3D2A7D2A6D2A5D251
:10429100B7900082E0D394FA400674FA900082F05D
:1042A1007E017F0090006CE012609990006BE02F1E
:1042B100FF50010E90001FEEF0A3EFF0EFD394FF3B
:1042C100EE940F400790001FE4F0A3F090006AE025
:1042D100700674FF90006AF074009000A9F09000DD
:1042E100BFE0D39402400674019000BFF09000C07B
:1042F100E07005756C028003756C039000C1E0D31A
:104301009401400674009000C1F09000C7E0C3948E
:104311000A5006740A9000C7F09000D1E07006744C
:10432100019000D1F09000D1E0B4FF0674FE90003E
:10433100D1F09000D8E0D394FE400674FE9000D8EE
:10434100F09000FEE0D39402400674019000FEF06C
:10435100900114E0D3940140067401900114F074AB
:10436100019000DEF074019000DFF074009000E62F
:10437100F07400900102F07400900106F07429902D
:1043810006BCF0742A9006C0F074179006C4F0744D
:104391001B9006D4F0741C9006D8F0D29C9000B10A
:1043A100E0D39404400674049000B1F09000E3E07F
:1043B100D39404400674049000E3F0E56FD39410A5
:1043C1004003756F109006BDE0D3940C4006740055
:1043D1009006BDF09006C1E0D3940C4006740090A5
:1043E10006C1F09006C5E0D3940C40067400900617
:1043F100C5F09006C9E0D3940C400674009006C93C
:10440100F09006CDE0D3940C400674009006CDF0F8
:104411009006D1E0D3940C400674009006D1F09040
:1044210006D5E0D3940C400674009006D5F09006B2
:10443100D9E0D3940C400674009006D9F09006DDC3
:10444100E0D3940C400674009006DDF09006E1E0A4
:10445100D3940C400674009006E1F0D2EC75CF01C4
:10446100A298B34005C298120616E54D6006A299BE
:10447100B3B340028005C299120AB4E54E640160EB
:1044810005E54EB4040280D5C28E7E107F00E5633F
:10449100126099E58D75F010A4FDACF0EF2DFDEEE5
:1044A1003CFCE58B75F01084FF7E00ED2FFFEC3EA8
:1044B100FE8E538F54D28E9000A3E060099000A32A
:1044C100E0C3943D4002805C9000171260A7900009
:1044D10017E0FEA3E0FF900019E0FCA3E0FDEFB5BB
:1044E1000542EEB5043EB21BA20DB3401975E700BB
:1044F100A21BB34008E5B54404F5B58006E5B55403
:10450100FBF5B575E710900019E0FEA3E0FF900000
:104511001BE0FCA3E0FDEF2DFDEE3CFC900019EC4F
:10452100F0A3EDF09000B0E060099000B0E0C3941A
:10453100034002806F1229C0A20DB350099000669A
:10454100E0C3942B4002800690009AE0F545E545D2
:1045510075F005A4FFAEF09007B8EEF0A3EFF09070
:104561000087E0C395604007E55EC3955F50079003
:1045710007B8E4F0A3F0AE2EAF2F9007B8E0FCA38C
:10458100E0FDEFD39DEE9C4004C2A1800B9000663C
:10459100E0C394415002D2A19000B0E0B40205A260
:1045A100A1B392A29000B0E0B4031C122ADBAE2E9C
:1045B100AF2F9007B8E0FCA3E0FDEFD39DEE9C4048
:1045C10004D2A18002C2A190008BE06009A2B330A5
:1045D1000F01B3B340028039A2B3300F01B34031B0
:1045E100A2B3301101B3401C9000BEE0B40306A297
:1045F1001EB3B3400280067404900045F0D21EA29F
:1046010011B3920FA211B330B301B34004A21192BE
:104611000FA2B6300E01B35003024C96A2B6300E73
:1046210001B35003024C96A2B6301001B3500302FD
:104631004ABA756D009000A3E0B43D1975E700A278
:1046410010B34008E5B554FBF5B58006E5B5440463
:10465100F5B575E710055DA212B3B35013AE53AFB4
:1046610054900008E0FCA3E0FDEDC39FEC9E4003E5
:104671000247BAE56CB4032EA227B34022E55DB42C
:104681002403756C01E55DC39424500690004574C4
:1046910001F0E55DD3942440067402900045F07565
:1046A1005D01D227805AE56CB40206756C01755D17
:1046B10024E55DB42405755D018045900045E070F9
:1046C10030E55DC3942450069000457401F0E55D2A
:1046D100D3942440067402900045F0E55DC3942410
:1046E1005002D222E55DD394244002D222C296C266
:1046F100959000C0E0B40105123B7A8003755D011D
:10470100AE55AF56AC53AD54EF2DFDEE3CFC7403EA
:10471100FF1260898C558D569000A3E060099000CE
:10472100A3E0C3943D40028043900017E0FEA3E064
:10473100FF9000A3E08E048F05FF12608974018C45
:10474100068D0712003990001BEEF0A3EFF09000E8
:104751001BE0F8A3E0900019C8F0A3C8F09000177F
:10476100E4F0A3F0C21BE5B554FBF5B5A2B4B34028
:1047710002C224A2A4B34002C223A2A3B34002C234
:1047810025A222B34002C222A21EB34006A2209259
:104791001F8002B21F90008BE06012E56C700EA2C8
:1047A1001EB35009A21F302001B3B340028006742A
:1047B10005900045F0C21E803AAE55AF56AC53ADE0
:1047C10054EF2DFDEE3CFC74018C068D071200396F
:1047D1008E558F56E56CC39402500DAC53AD547495
:1047E10088C39D74139C40028009123B7A74069021
:1047F1000045F0E55DB424127403900045F0D22227
:104801009000C0E0B40103123B7AAE57AF58AC53ED
:10481100AD54EF2DFDEE3CFC8C578D58AE53AF548B
:10482100EFD39DEE9C401190000FE0FAA3E0FBEB6B
:10483100C394E8EA94034002800690000F1260A737
:1048410090000CE0FEA3E0FFAC53AD54EF2DFDEE64
:104851003CFC90000CECF0A3EDF09000C0E0B40142
:104861001DAE53AF54740512609974038E048F0505
:10487100FF126089900008ECF0A3EDF08016AE53B2
:10488100AF5474031260997401120039900008EE5C
:10489100F0A3EFF0C28E758D00758B007563007506
:1048A1005401755300D28EE55D240875F00984AF7B
:1048B100F07E00EF4E707590000CE0F8A3E09000E0
:1048C1000AC8F0A3C8F090000AE0FEA3E0FFEF4E93
:1048D100600B7C7B7D89125F878E518F5290000C1B
:1048E100E4F0A3F0AE51AF527428BE00039F501004
:1048F100E5622FFF50010E74011200398E518F5263
:104901008552629000C7E0A851B8000DD39552407E
:1049110008E552900044F080099000C7E01490002F
:1049210044F0E56C60067552007551009000BEE0E0
:10493100B4030890003DE0655D6002800BA21FB3E7
:104941004004D2218002B221E55D640B6005E55D82
:10495100B41D099000B0E0600312202B900042E0EA
:10496100655D6007900043E0B55D03756E00A213BD
:10497100B35006A212B3B34003024A2290007CE076
:10498100B401739000FEE0B40214120C5590006F54
:10499100E075F0BEA4FFAEF08E5B8F5C8056E566DD
:1049A10075F00A84FF7E009005761260C0E0F55A2A
:1049B100755900AE59AF5A9000A1E0126099746424
:1049C1008E048F05FF1260898C5B8D5CE55C900025
:1049D1000EF0AE59AF5A90007AE012609974648E6D
:1049E100048F05FF12608974BE8C068D07126099D1
:1049F1008E5B8F5C801790007AE075F0BEA4FFAEED
:104A0100F08E5B8F5C9000A1E090000EF0E560C33A
:104A110094CC500690007AE070028003123C4ED292
:104A210013E56CB40106E55D640B60028009756FE6
:104A3100019000467401F0E56C70799000C3E0606C
:104A41000D90006EE0A851B80006955240028038E2
:104A51009000C3E0B4021790003BE0655D600790F1
:104A6100003CE0B55D03756F03756B00800CC200FF
:104A7100756B00900015E4F0A3F090006EE0600605
:104A81007409900045F0802C90003BE0655D600763
:104A910090003CE0B55D03756F0190003BE0B55DB2
:104AA100069000467401F090003CE0B55D0674028A
:104AB100900046F0A210B3920EA210B330B601B32B
:104AC1005003024C96756D019000A3E0B43D197539
:104AD100E700A210B34008E5B54404F5B58006E54A
:104AE100B554FBF5B575E710E5B54401F5B5742B83
:104AF100900066F0A210920EE55DD3944A4014D264
:104B010012E55DD3946E400B7404900045F0D222FF
:104B1100755D469000CBE0B40107E569C39414408C
:104B2100028009123B7A7413900045F0A2293003E8
:104B310001B3501D75E700A229B34008E5B544084B
:104B4100F5B58006E5B554F7F5B575E710A22992DC
:104B510003A22A300401B3501D75E700A22AB34015
:104B610008E5B54402F5B58006E5B554FDF5B57522
:104B7100E710A22A9204A22B300501B3500FA22BF9
:104B8100B34004D2A08002C2A0A22B9205A22C3075
:104B91000601B3500FA22CB34004D2978002C297F2
:104BA100A22C9206A22D300701B3500FA22DB340C3
:104BB10004D2A28002C2A2A22D9207A22E30080125
:104BC100B3500FA22EB34004D2A18002C2A1A22EE3
:104BD1009208A22F300901B3501D75E700A22FB32F
:104BE1004008E5B54440F5B58006E5B554BFF5B5D7
:104BF10075E710A22F9209A230300A01B3501D753A
:104C0100E700A230B34008E5B54480F5B58006E57C
:104C1100B5547FF5B575E710A230920AA231300B79
:104C210001B3500FA231B34004D2878002C287A2E0
:104C310031920BA232300C01B3500FA232B34004B7
:104C4100D2908002C290A232920CE569C394415085
:104C510009740E900045F0123B7A90004DE0FE90F1
:104C61000049E004C39E4009900049E0D394064006
:104C71000974FB900045F0123B7A900052E06015F8
:104C8100900052E0FE90004CE06E600974FE9000CE
:104C910045F0123B7AA222B34004C296C29590001D
:104CA100FBE0600CAE51AF527414BE00059F400290
:104CB1008048900083E0905915F8282873803BA222
:104CC100B4B35005A224B340028005123CA6D224FD
:104CD1008028A2A3B35005A225B340028005123C4F
:104CE100A6D2258015A2A4B35005A223B340028009
:0A4CF10005123CA6D22380028000C9
:10591500024CBE024CC0024CD3024CE6024CF902CA
:025925004CFB39
:104CFB00A215B3B3500890003DE0655D6003024D13
:104D0B00DAA201B35006A200B3B34003024DD69012
:104D1B0000BEE0B403028003024DABA20DB34067AB
:104D2B00A221B3402D12363AE55CF5FBE55BF5FCB1
:104D3B00D293A202B34002D2879000DCE0B40210FF
:104D4B00123667E55CF5FBE55BF5FC75A700D287D2
:104D5B00803312363AE55CF5EBE55BF5ECD291A2CC
:104D6B0002B34006E5B54410F5B59000DCE0B402A3
:104D7B0014123667E55CF5EBE55BF5EC75A700E522
:104D8B00B54410F5B5801712363AE55CF5FBE55BDB
:104D9B00F5FCE55CF5EBE55BF5ECD293D291802B62
:104DAB0012363AE55CF5FBE55BF5FCD293A202B358
:104DBB004002D2879000DCE0B40210123667E55C4B
:104DCB00F5FBE55BF5FC75A700D287C215D216A2E1
:104DDB0016B3B3500890003EE0655D6003024EB918
:104DEB00A201B35006A200B3B34003024EB590002C
:104DFB00BEE0B403028003024E8AA20DB34067A249
:104E0B0021B3402D12363AE55CF5E9E55BF5EAD2C4
:104E1B0094A202B34002D2909000DCE0B4021012D4
:104E2B003667E55CF5E9E55BF5EA75A700D290809E
:104E3B003312363AE55CF5EDE55BF5EED292A20264
:104E4B00B34006E5B54420F5B59000DCE0B40214A0
:104E5B00123667E55CF5EDE55BF5EE75A700E5B59C
:104E6B004420F5B5801712363AE55CF5E9E55BF5BC
:104E7B00EAE55CF5EDE55BF5EED294D292802B1270
:104E8B00363AE55CF5E9E55BF5EAD294A202B3406C
:104E9B0002D2909000DCE0B40210123667E55CF5AC
:104EAB00E9E55BF5EA75A700D290D215C216E56F5E
:0E4EBB00905927F82828730252E89000E3E08F
:06592700024EC2024EC553
:104EC90090595AF8282873121B078012121B078061
:0E4ED9000D121B918008121C3D8003121C3D1F
:0F595A00024ED0024ED5024EDA024EDF024EE46C
:104EE700756F020252E8121D69121E80A237B34085
:104EF700229000A5E0F56B900076E0256BFE900010
:104F070044E075F01E84FC7F00EE2CF5347410909D
:104F17000045F09007AEE0FEA3E0FF740A12609927
:104F270090000AE0FCA3E0FD74098F02FF1260897C
:104F37008D078C038E048A058B06125F879007B254
:104F4700EEF0A3EFF09000CCE0B401087478BE0057
:104F5700059F4002800D74789007B2F8E4F0E8A34B
:104F6700F0801B9007B2E0FEA3E0FF74F0BE0003E1
:104F77009F500B74F09007B2F8E4F0E8A3F0E53423
:104F870070037534019007B2E0FEA3E0FFE5342F0C
:104F9700FF50010E9007B2EEF0A3EFF0756F03908C
:034FA7000046E0E1
:03592D00024EED3A
:104FAA00905969F82828738010A2384003756F0A4F
:094FBA008007A2384003756F0B5B
:09596900024FB1024FB3024FBC22
:104FC3000252E89006BDE060031221149000FCE059
:104FD300B401149000FDE0A851B8000495525007A5
:104FE300E55EC3955F400280030250709000B1E01C
:104FF300D39402403F900085E02403A851B80004F5
:1050030095525009900087E0D3956050028008D2F2
:10501300017408900045F0900085E0A851B80005A0
:10502300D39552500B900087E02403C39560500240
:10503300C2018039900085E02403A851B80004958B
:10504300525007E55EC3955F40028008D2017408A1
:10505300900045F0900085E0A851B80005D3955223
:105063005009E55F240FC3955E5002C2019000CB47
:10507300E07007E569C3941440028002D201A201E3
:105083004005756F04800A756F10900015E4F0A356
:10509300F0A20DB34029E56675F00A84FF7E009007
:1050A30005761260C0E0C394695005122060800F3A
:1050B3009007B0E0F8A3E09007AEC8F0A3C8F002F1
:0650C30052E89000B1E08C
:06593000024FC60250C543
:1050C900905972F8282873120D3F8012120D3F80F3
:0E50D9000D120EED8008120F9F8003120F9F24
:0F5972000250D00250D50250DA0250DF0250E44A
:1050E7009006C1E060031221F0756F050252E812C5
:1050F70010AB756F069006C5E060031222E09006BC
:10510700C9E060031223BC0252E890000EE060067B
:10511700A20DB3B34002801D90000EE02529FFAE1B
:105127002850010E8E288F29E55DD39412500690E2
:10513700000EE014F01212F1756F079006CDE060D3
:10514700031224989006D1E060031225740252E8F6
:105157009000FEE0B40203120CCD12154E756F08D5
:105167009006D5E060031226509006D9E06003123E
:10517700272C0252E812190AA215B35005A216B33A
:1051870040028004D215D216756F109006DDE060DC
:10519700031228089006E1E060031228E40252E8AF
:1051A7000252E8900035E0C394465008C296744610
:1051B700900035F090003FE0B4011DE534240AF576
:1051C700349007B2E0FEA3E0FF740A2FFF50010EF0
:1051D7009007B2EEF0A3EFF085345A7559009000AE
:1051E7003BE0F5721236B2E55C900035F0900004B2
:1051F700E559F0A3E55AF0E572900036F0C2189031
:1052070007B2E0F559A3E0F55A90003BE0F57212BA
:1052170036B2E55C900033F0900000E559F0A3E565
:105227005AF0E572900034F0C217E56CB4010575C9
:105237006F0B8003756F030252E8900039E0C39447
:105247004650139000CCE0B40104C2968002C29588
:105257007446900039F0900040E0B4011DE5342415
:105267000AF5349007B2E0FEA3E0FF740A2FFF505F
:10527700010E9007B2EEF0A3EFF085345A7559008E
:1052870090003CE0F5721236B2E55C900039F09080
:105297000006E559F0A3E55AF0E57290003AF0C22E
:1052A7001A9007B2E0F559A3E0F55A90003CE0F5F3
:1052B700721236B2E55C900037F0900002E559F0C3
:1052C700A3E55AF0E572900038F0C219E56CB40115
:1052D70003756C00756F0380088006800480028068
:0152E70000C6
:105936000250F602511102515702517C0251A70240
:1059460051AA0252410252E00252E20252E40252CB
:04595600E60252E82B
:1052E800900033E0B55D73A217404F900000E0FED8
:1052F800A3E0FFEF4E6021AE55AF56900000E0FCF2
:10530800A3E0FD120003740A8E048F05FF12608962
:10531800900000ECF0A3EDF0900034E0601A9000EB
:1053280000E0FEA3E0FFAC55AD56EF2DFDEE3CFCD2
:10533800900000ECF0A3EDF0D217AE53AF549000FC
:1053480000E0FCA3E0FDEFC39DEE9C400D123CF392
:10535800D296C21774C8900033F0A217B3B350079F
:10536800900033E0B55D02800D123CF3D29674C80C
:10537800900033F0C217900035E0B55D70A2184078
:105388004F900004E0FEA3E0FFEF4E6021AE55AF62
:1053980056900004E0FCA3E0FD120003740A8E049A
:1053A8008F05FF126089900004ECF0A3EDF09000E7
:1053B80036E0601A900004E0FEA3E0FFAC55AD565D
:1053C800EF2DFDEE3CFC900004ECF0A3EDF0D218BC
:1053D800AE53AF54900004E0FCA3E0FDEFC39DEE94
:1053E8009C400AC2967446900035F0C218A218B3C1
:1053F800B35007900035E0B55D02800AC296744646
:10540800900035F0C218900037E0B55D7EA21940D3
:105418004F900002E0FEA3E0FFEF4E6021AE55AFD3
:1054280056900002E0FCA3E0FD120003740A8E040B
:105438008F05FF126089900002ECF0A3EDF0900058
:1054480038E0601A900002E0FEA3E0FFAC55AD56CC
:10545800EF2DFDEE3CFC900002ECF0A3EDF0D2192C
:10546800AE53AF54900002E0FCA3E0FDEFC39DEE05
:105478009C4018123CF39000CCE0B40104D2968012
:1054880002D295C21974C8900037F0A219B3B3506C
:1054980007900037E0B55D028018123CF39000CC0D
:1054A800E0B40104D2968002D29574C8900037F017
:1054B800C219900039E0B55D7BA21A404F900006F2
:1054C800E0FEA3E0FFEF4E6021AE55AF5690000618
:1054D800E0FCA3E0FD120003740A8E048F05FF129E
:1054E8006089900006ECF0A3EDF090003AE0601AB5
:1054F800900006E0FEA3E0FFAC55AD56EF2DFDEEA3
:105508003CFC900006ECF0A3EDF0D21AAE53AF5479
:10551800900006E0FCA3E0FDEFC39DEE9C401590D3
:1055280000CCE0B40104C2968002C2957446900093
:1055380039F0C21AA21AB3B35007900039E0B55D2A
:105548000280159000CCE0B40104C2968002C29596
:105558007446900039F0C21A9000CEE0B40202807E
:105568000302567C900068E0D3956550649000680B
:10557800E0F4042565FE9000D1E08E00F5F0E884A3
:10558800FF7E008F72EFC39410500CEF8572F0A469
:10559800FDACF08D7280037572FF900068E0D395C2
:1055A80072400B900068E0C39572F57080037570C7
:1055B800009000ECE0D3957040069000ECE0F570A8
:1055C8009000EDE0C3957050069000EDE0F5708016
:1055D80071900068E0C39565FE9000D1E08E00F5FB
:1055E800F0E884FF7E008F72EFC39410500CEF85B3
:1055F80072F0A4FDACF08D7280037572FF85725A4B
:10560800755900900068E0255AFFAE5950010E8E7A
:10561800598F5A74FFBE0009D39F4005855A708080
:10562800037570FF9000ECE0D3957040069000EC95
:10563800E0F5709000EDE0C3957050069000EDE045
:10564800F570A20DB3B3500D900069E0FE9000D93B
:10565800E0D39E5002800A7407900045F0C29780FC
:105668001375A710E5CDC395704004C2978002D288
:105678009775A700E56EC39409500AA2EDB34005DB
:10568800C2ED122C7AAE53AF547410C39F74279E88
:10569800400C900067E0C3945A40030258EEA212EF
:1056A800B34009123B7A7406900045F0A21DB3403E
:1056B80008E5B54404F5B58006E5B554FBF5B5A293
:1056C80014B3500EE560D394334007E560C394CC1F
:1056D8004002802FE5B54401F5B5742B900066F0C3
:1056E80090007AE075F0BEA4FFAEF08E5B8F5C741C
:1056F80002BE000AD39F4006755C02755B00123C2F
:105708004ED214900067E0D394014007E560C3943B
:105718001A40028002C2149006BDE06003122114F0
:10572800A229300301B35017A229B34008E5B544B4
:1057380008F5B58006E5B554F7F5B5A229920390AA
:1057480006C1E060031221F0A22A300401B3501709
:10575800A22AB34008E5B54402F5B58006E5B5547C
:10576800FDF5B5A22A92049006C5E060031222E076
:10577800A22B300501B3500FA22BB34004D2A08056
:1057880002C2A0A22B92059006C9E060031223BCB6
:10579800A22C300601B3500FA22CB34004D297803C
:1057A80002C297A22C92069006CDE06003122498BC
:1057B800A22D300701B3500FA22DB34004D2A2800E
:1057C80002C2A2A22D92079006D1E06003122574AE
:1057D800A22E300801B3500FA22EB34004D2A180EC
:1057E80002C2A1A22E92089006D5E06003122650AC
:1057F800A22F300901B35017A22FB34008E5B544D2
:1058080040F5B58006E5B554BFF5B5A22F920990CD
:1058180006D9E0600312272CA230300A01B35017D2
:10582800A230B34008E5B54480F5B58006E5B55427
:105838007FF5B5A230920A9006DDE06003122808D1
:10584800A231300B01B3500FA231B34004D287808C
:1058580002C287A231920B9006E1E060031228E4AD
:10586800A232300C01B3500FA232B34004D2908060
:1058780002C290A232920C900067E0C3945A501072
:10588800E56EB40909900067E004F0756E00803B8E
:10589800E56EB40903756E00755400755300758D77
:1058A80000758B00756300900066E0C39441500852
:1058B800900066E004F080067441900066F0900065
:1058C80066E0B44106E5B554FEF5B5900067E0D34F
:1058D80094014007E569C3944140028009740E9021
:0958E8000045F0123B7A02445E17
:105981000000010001400160018001A001C001E0AF
:1059910002000300039603B603D603F404000500D6
:1059A1000512052405360548055A056C057E059046
:1059B10005A805C005DE0600061406280646066E83
:1059C10006AE00FF013F015F017F019F01BF01DFC3
:1059D10001FF02FF039503B503D503F303FF04FFA2
:1059E10005110523053505470559056B057D058F0E
:1059F10005A705BF05DD05F1061306270645066D5A
:105A010006AD06ED0FAA0FA50F9F0F9A0F940F8DEC
:105A11000F870F800F780F710F680F600F570F4EB0
:105A21000F450F3B0F300F250F1A0F0E0F020EF50A
:105A31000EE80EDB0ECC0EBE0EAE0E9F0E8E0E7D50
:105A41000E6C0E5A0E470E340E200E0C0DF70DE2A1
:105A51000DCB0DB50D9D0D850D6D0D540D3A0D2020
:105A61000D050CE90CCE0CB10C940C760C580C3ACB
:105A71000C1B0BFB0BDB0BBB0B9A0B790B570B3581
:105A81000B130AF10ACE0AAB0A870A640A400A1C00
:105A910009F809D409B0098C09670943091F08FBF2
:105AA10008D608B2088E086A0846082307FF07DCF3
:105AB10007B9079607730751072F070D06EC06CAAA
:105AC10006AA068906690649062A060A05EC05CDD5
:105AD10005B0059205750558053C0520050504EA44
:105AE10004CF04B5049C04820469045104390422DE
:105AF100040B03F403DE03C803B2039D038903759A
:105B01000361034D033B03280316030402F202E180
:105B110002D102C002B002A00291028202730265A8
:105B210002570249023C022F02220216020901FD1C
:105B310001F201E601DB01D001C601BB01B101A700
:105B4100019D0194018B018201790170016801605D
:105B5100015801500148014101390132012B012550
:105B6100011E01180111010B010500FF00FA0FA62A
:105B71000FA00F990F920F8B0F840F7C0F740F6B77
:105B81000F620F580F4E0F430F380F2C0F1F0F12BC
:105B91000F050EF70EE80ED80EC80EB70EA50E9320
:105BA1000E800E6C0E580E420E2C0E150DFD0DE4DE
:105BB1000DCB0DB10D950D790D5D0D3F0D200D0135
:105BC1000CE10CC00C9E0C7C0C590C350C100BEA32
:105BD1000BC40B9E0B760B4F0B260AFD0AD40AAAA7
:105BE1000A800A550A2A09FF09D409A8097C095023
:105BF100092508F908CD08A10875084A081E07F308
:105C010007C8079D07730749072006F706CE06A6B2
:105C1100067E06570630060A05E405BF059B057793
:105C210005540532051004EF04CE04AE048F04714F
:105C310004530435041903FD03E203C703AD0394C0
:105C4100037B0363034B0334031E030802F302DEE9
:105C510002CA02B602A30291027F026D025C024CEB
:105C6100023C022C021D020E020001F201E401D7E6
:105C710001CA01BE01B101A6019A018F0185017A14
:105C810001700166015D0153014A01410139013190
:105C91000129012101190112010B010400FD00F785
:105CA10000F000EA00E400DE00D900D300CE00C914
:105CB10000C400BF00BA00B500B100AD00A800A447
:105CC10000A0009C009900950091008E008A008739
:085CD10000840081007E007BCD
:10009E007547009007BAE4F0A3F075310075300093
:1000AE00754D00754E00C234D23574FE9007C4F8FB
:1000BE00E4F0E8A3F074FE9007C6F8E4F0E8A3F0CD
:1000CE00745A9007C8F0745A9007C9F0D236C228F5
:1000DE00C238C23322750B00750A00AE0AAF0BACE4
:1000EE0008AD09EDC39FEC9E401674FF1260797542
:1000FE00CF01780B740126F6500418E436F650DB67
:10010E0022900041E0B4AA1C900776E0B43C159012
:10011E0007B6E0FEA3E0FFEF4E6009741EBE0004BA
:10012E00D39F500302023D755C00755B0075F809A4
:10013E009007B6E0FEA3E0FF74076F4E6006740EE4
:10014E006F4E7006743A900776F09007B6E0FEA3F5
:10015E00E0FF7408BE001ED39F401A7E017F0890F8
:10016E0007B6E0FCA3E0FD1DBDFF011C1200038ECF
:10017E00598F5A801F9007B6E0FEA3E0FF74081255
:10018E0060DD8F048E057E017F08CDCCCD1200037D
:10019E008E598F5AAE5BAF5C740CD39F74019E5018
:1001AE0003020238A2F9B3407EE55C455B7003752D
:1001BE00A382AE5BAF5C74016F4E700375A300AE8D
:1001CE005BAF5C74026F4E700D9007B7E075F00276
:1001DE00A4FDACF08DA3AE5BAF5C74036F4E7003E9
:1001EE0075A300AE5BAF5C7403BE00039F5013ACEF
:1001FE0059AD5AED2FFFEC3EFE9000721260C0E03A
:10020E00F5A3AE5BAF5CEFB40B09EEB4010574144D
:10021E00126079AE5BAF5CEFB40B07EEB401037501
:10022E00F80D785B1260ED0201A2900041E4F0221D
:10023E00755C00755B0075F8099007B6E0FEA3E0EB
:10024E00FF7408BE001ED39F401A7E017F089007E0
:10025E00B6E0FCA3E0FD1DBDFF011C1200038E598C
:10026E008F5A801F9007B6E0FEA3E0FF740812605D
:10027E00DD8F048E057E017F08CDCCCD1200038E5E
:10028E00598F5AAE5BAF5C7411D39F74019E5003AD
:10029E0002036EA2F9B3500302036BE55C455B707B
:1002AE000375A3D2AE5BAF5C74016F4E700375A382
:1002BE0000AE5BAF5C74026F4E700D9007B7E075C9
:1002CE00F002A4FDACF08DA3AE5BAF5C74036F4E79
:1002DE00700375A300AE5BAF5C74046F4E70037554
:1002EE00A300AE5BAF5C74056F4E700375A300AEDA
:1002FE005BAF5C74066F4E700375A300AE5BAF5CB4
:10030E0074076F4E700375A300AE5BAF5C74086F1D
:10031E004E700375A300AE5BAF5C7408BE00039F06
:10032E005016AC59AD5AED2FFFEC3EFE90006D12FB
:10033E0060C0E5A3F075A300AE5BAF5CEFB410092F
:10034E00EEB401057414126079AE5BAF5CEFB410BD
:10035E0007EEB4010375F80D785B1260ED020291A1
:10036E0022755C00755B0075F809AE5BAF5C7417A7
:10037E00BE0004D39F5003020447A2F9B3500302F8
:10038E000444E55C455B700375A3D2AE5BAF5C7451
:10039E00016F4E700375A300AE5BAF5C74026F4EBF
:1003AE00700D9007B7E075F002A4FDACF08DA3AE12
:1003BE005BAF5C74036F4E700375A300AE5BAF5CF6
:1003CE0074046F4E700375A300AE5BAF5C74056F63
:1003DE004E700375A300AE5BAF5C74066F4E700378
:1003EE0075A300AE5BAF5C74076F4E700375A30010
:1003FE00AE5BAF5C74086F4E700375A300AE5BAF5F
:10040E005C7408BE00039F500C90004F1260C0E554
:10041E00A3F075A300AE5BAF5C74166F4E700574DF
:10042E0014126079AE5BAF5C74166F4E700375F884
:10043E000D785B1260ED02037822900041E0B4ABC0
:10044E000280030204E2755C00755B0075F809AE6C
:10045E005BAF5C7412BE007CD39F4078A2F9B340B0
:10046E0070E55C455B700375A382AE5BAF5C740197
:10047E006F4E700375A300AE5BAF5C74026F4E706F
:10048E000D9007B7E075F002A4FDACF08DA3AE5B46
:10049E00AF5C74036F4E700375A300AE5BAF5C74FC
:1004AE0003BE00039F50099000541260C0E0F5A3F4
:1004BE00AE5BAF5C74116F4E70057414126079AE42
:1004CE005BAF5C74116F4E700375F80D785B126044
:1004DE00ED02045D229007C1E4F074649007B6F853
:1004EE00E4F0E8A3F012036F74C89007B6F8E4F0D6
:1004FE00E8A3F090005BE0B4371A900058E090004B
:10050E004FF0900059E0900050F090005AE09000AB
:10051E0051F080469007C17401F074659007B6F8EB
:10052E00E4F0E8A3F012036F74C89007B6F8E4F095
:10053E00E8A3F090005BE0B4371A900058E090000A
:10054E004FF0900059E0900050F090005AE090006B
:10055E0051F0800674029007C1F09007C2E4F07467
:10056E00669007B6F8E4F0E8A3F012036F74C89033
:10057E0007B6F8E4F0E8A3F090005AE0B437129012
:10058E000058E0900049F0900059E0900052F08041
:10059E00769007C27401F074679007B6F8E4F0E83D
:1005AE00A3F012036F74C89007B6F8E4F0E8A3F056
:1005BE0090005AE0B43712900058E0900049F09045
:1005CE000059E0900052F0803E74029007C2F07421
:1005DE00689007B6F8E4F0E8A3F012036F74C890C1
:1005EE0007B6F8E4F0E8A3F090005AE0B4371290A2
:1005FE000058E0900049F0900059E0900052F080D1
:10060E000674039007C2F022E54E64046006E59975
:10061E0064FF6002802AA2344004D2348020E54E6A
:10062E00600874E6254E900045F0754E00E54D606D
:10063E000874F0254D900045F0754D00C2348002CF
:10064E00C234E54E9033F8F8282873754E00E599BC
:10065E00B4FF03754D01E599B4FE03754D02E5999E
:10066E00B4FD03754D03E599B4FC03754D04E5998E
:10067E00B4FA03754D05E599B4FB06754E01123BB0
:10068E007AE599B4F906754E04123B7AE599D3943E
:10069E00E54007E599C394F04002801685994F75A1
:1006AE004E027E017F00E54FC394E61260998E32B2
:1006BE008F339007BAE4F0A3F0E599D394C44007C2
:1006CE00E599C394E64002802885994F754E0374D0
:1006DE00E5C3954FF533753200AE32AF3390598185
:1006EE00126068E493F87401939007BAC8F0A3C837
:1006FE00F0D299020AB3900058E070429007BAE027
:10070E00FEA3E0FF74FFBE00039F5009EFC39446A3
:10071E00EE940640119007BAE0FEA3E0FFEFD394EB
:10072E006DEE940640139007BAE0FEA3E0FF900032
:10073E00761260C0E599F080038599738011900759
:10074E00BAE0FEA3E0FF9000761260C0E599F0904B
:10075E0007BA1260A79007BAE0FEA3E0FFEFB4015C
:10076E0006EEB40702800302089B900776E0B43CC5
:10077E00028003020885C29C900058E0900114F09C
:10078E00900059E0900083F090005AE09000A3F0A2
:10079E0090005BE09000CCF090005CE0900078F070
:1007AE0090005DE09000BEF090005EE09000DCF006
:1007BE0090005FE09000B0F0900060E09000CEF00E
:1007CE00900061E09000FEF012373490006AE090E5
:1007DE0000E5F090006BE090009CF090006CE090D3
:1007EE00009DF074639007B6F8E4F0E8A3F074ABE4
:1007FE00900041F0120448900041E4F075096475D0
:10080E0008001200E3A21C4038757201E572D39401
:10081E0007502CE5729007B6F8E4F0E8A3F074AA3E
:10082E00900041F012010FE572C39407500975094B
:10083E00647508001200E37872740126F650CD80BC
:10084E0036757208E572D3940E502CE5729007B689
:10085E00F8E4F0E8A3F074AA900041F012010FE55D
:10086E0072C3940E50097509647508001200E3787E
:10087E0072740126F650CD74C89007B6F8E4F0E80D
:10088E00A3F0D29C754E00754D007599FB020AB30C
:10089E009007BAE0FEA3E0FFEF4E70068599317522
:1008AE0030009007BAE0FEA3E0FF74016F4E701B9C
:1008BE00AC30AD31AA32AB33ED2BFBEC3AFA8A06F3
:1008CE008B079000761260C0E599F09007BA12601F
:1008DE00A79007BAE0FEA3E0FF74026F4E7021AC42
:1008EE0030AD3174566D4C7006E54F64E660028093
:1008FE0003123B7A123734854F99754E00754D00B1
:10090E00020AB39007BAE0FEA3E0FF9000761260F1
:10091E00C0E599F09007BA1260A79007BAE0FEA35F
:10092E00E0FFAC32AD338F028E038C068D079059EB
:10093E00C3126068E493F9740193FEEAD39EEB99B7
:10094E004009854F99754E00754D00020AB3900708
:10095E00BAE0FEA3E0FF9000761260C0E599F09039
:10096E0007BA1260A79007BAE0FEA3E0FFEFB4004B
:10097E0006EEB401028003020AB3900051E075F056
:10098E0002A4FDACF08D72ED9000761260CBEDFA04
:10099E00E0FBEA9000791260CBEBFAE0FBEA2BFA6F
:1009AE00900051E0B502028003020AA50DED900001
:1009BE00761260CBE572FDE0FAED90007A1260CB14
:1009CE00EAFDE0FAEDC39AFD900051E0B505028014
:1009DE0003020AA5E5729000781260CBE572FDE085
:1009EE00FAED90007B1260CBEAFDE0FAED2AFD9065
:1009FE000051E0B505028003020AA5E57290007C65
:100A0E001260CBFDE0FAED900051E0F4042A900064
:100A1E0058F0E57290007D1260CBFDE0FAED90008B
:100A2E0051E0F4042A900059F0E57290007E1260B5
:100A3E00CBFDE0FAED900051E0F4042A90005AF05C
:100A4E00E57290007F1260CBFDE0FAED900051E070
:100A5E00F4042A9007B6F8E4F0E8A3F074AB900023
:100A6E0041F01204487509647508001200E39007FE
:100A7E00B61260A71204487509647508001200E3E7
:100A8E009007B61260A71204487599F97509647536
:100A9E0008001200E380FE7599FF75096475080061
:050AAE001200E380FED0
:0F33F80002065902070402089E02091102095C2D
:100AB30022E54D903407F8282873020B989007BA63
:100AC300E0FEA3E0FF9000471260C0E0F5999007B5
:100AD300BA1260A79007BAE0FEA3E0FF74116F4E4D
:100AE3007003754D00020B98856D99020B98900762
:100AF300BAE0FEA3E0FF9000761260C0E0F599EF44
:100B0300B40107EEB40703754D009007BA1260A74E
:070B1300020B989007BBE004
:0F340700020ABD020AC0020AEB020AF1020B160A
:100B1A009035BAF82828738552998067855E99803E
:100B2A0062856099805D856499805885669980534D
:100B3A00856799804E85689980498569998044902E
:100B4A000016E0F599803CA235B340077599FAC2C0
:100B5A00358017A226B3400575990F800B90004582
:100B6A00E0F599900045E4F0C2268017856A9980DD
:100B7A0012856599800D856B9980087599FC8003AB
:030B8A00754D00A6
:1035BA00020B21020B26020B2B020B30020B3502E7
:1035CA000B3A020B3F020B44020B49020B51020B4E
:0D35DA0076020B7B020B80020B85020B8A30
:0B0B8D009007BA1260A780031235E742
:03341600020B9511
:100B980022E537255AFFAE5950010E9000761260B3
:100BA800C0E0F538E537255AFFAE5950010E0FBFA2
:100BB80000010E9000761260C0E0F539853F3BE5F4
:100BC80038B539058538378041E539D39538401D22
:100BD800E539C39538853AF0A4FFAEF0E53B8E04BD
:100BE8008F05FF126089ED2538F537801DE538C37C
:100BF8009539853AF0A4FFAEF0E53B8E048F05FFEA
:100C0800126089EDF4042538F53722E539D3953893
:100C1800401DE539C39538853AF0A4FFAEF0E53BB1
:100C28008E048F05FF126089ED2538F537801DE5A4
:100C380038C39539853AF0A4FFAEF0E53B8E048FB2
:100C480005FF126089EDF4042538F5372290007C01
:100C5800E0B40170E56675F00A84FF7E008F37E521
:100C68006675F00A84ADF07C008D3A753F0A7559B7
:100C780005755A24E537C394115005120B9980065F
:100C88009005ABE0F537E53790006FF0E56675F055
:100C98000A84FF7E008F37E56675F00A84ADF07C24
:100CA800008D3A753F0A755905755A5AE537C39448
:100CB800115005120B9980069005E1E0F537E537EC
:100CC80090000EF02290007CE0B4016AE56675F0B1
:100CD8000A84FF7E008F37E56675F00A84ADF07CE4
:100CE800008D3A753F0A755905755A36E537C3942C
:100CF800115005120B9980069005BDE0F537853730
:100D08004BE56675F00A84FF7E008F37E56675F05F
:100D18000A84ADF07C008D3A753F0A755905755AFD
:100D280048E537C394115005120B9980069005CFFA
:100D3800E0F53785374C22E55E75F00484FF7E00C8
:100D48008F37E55E75F00484ADF07C008D3A753F11
:100D580004755901755A00E537C3943F5005120BC5
:100D68009980069001B5E0F53785372975280090F8
:100D78000044E075F020A4FFAEF09000C7E08E04B8
:100D88008F05FF1260898D379000AFE0D3955E50D4
:100D980003020E459000D3E0D3955E4010ED90011C
:100DA800B61260CBE0F52B752A00020E4290009E29
:100DB800E0D3955E4043E5379001B61260CBE0F58D
:100DC80038E5379001D61260CBE0F5399000D3E0D2
:100DD800F404255EF53A90009EE0FE9000D3E0F41E
:100DE800042EF53BE538B539058538378003120CF4
:100DF8001385372B752A008041E5379001D612609C
:100E0800CBE0F538E5379001F61260CBE0F5399084
:100E1800009EE0F404255EF53A9000AFE0FE9000F5
:100E28009EE0F4042EF53BE538B539058538378062
:100E380003120C1385372B752A00020EEC9000D68E
:100E4800E0D3955E5011E5379002361260CBE0F59D
:100E58002B752A00020EEC90009FE0D3955E50435C
:100E6800E5379002161260CBE0F538E53790023688
:100E78001260CBE0F53990009FE0F404255EF53A66
:100E88009000D6E0FE90009FE0F4042EF53BE53894
:100E9800B539058538378003120C1385372B752A29
:100EA800008041E5379001F61260CBE0F538E53770
:100EB8009002161260CBE0F5399000AFE0F40425FB
:100EC8005EF53A90009FE0FE9000AFE0F4042EF546
:100ED8003BE538B539058538378003120C1385375B
:100EE8002B752A00229000E7E0F53C753F117559F3
:100EF80002755A00AE51AF52E53C75F00FA4FDAC37
:100F0800F0EDD39FEC9E4021E53C8E048F05FF1247
:100F18006089ED75F010A4FFAEF0E55E75F0118400
:100F2800FD7C00ED2FF53D800EE55E75F01184FF28
:100F38007E00EF24F0F53D853D37E55E75F01184C0
:100F4800AFF07E008F3A120B9985373EAE51AF5203
:100F58009000E7E075F00FA4FDACF0EDD39FEC9E98
:100F68004028755902755A10853D37120B99853EF0
:100F780038853739AE51AF52E53C8E048F05FF12E4
:100F880060B48D3A853C3B120C13853729752800CF
:100F9800752B64752A00229000E7E0F53C753F1137
:100FA800755902755A00AE51AF52E53C75F00FA461
:100FB800FDACF0EDD39FEC9E4021E53C8E048F05FF
:100FC800FF126089ED75F010A4FFAEF0E56075F0D2
:100FD8001184FD7C00ED2FF53D800EE56075F01164
:100FE80084FF7E00EF24F0F53D853D37E56075F020
:100FF8001184AFF07E008F3A120B9985373EAE51BF
:10100800AF529000E7E075F00FA4FDACF0EDD39F70
:10101800EC9E4028755902755A10853D37120B9978
:10102800853E38853739AE51AF52E53C8E048F0581
:10103800FF1260B48D3A853C3B120C138537297535
:1010480028009000B1E0B40453E55E75F00484FF15
:101058007E008F37E55E75F00484ADF07C008D3A34
:10106800753F04755901755A00E537C3943F50051B
:10107800120B9980069001B5E0F537AE28AF29E547
:101088003712609974648E048F05FF126089AE2848
:10109800AF29EF2DFDEE3CFC8C288D29752B64754E
:1010A8002A002290007CE0B40146E56675F00A84C7
:1010B800FF7E008F37E56675F00A84ADF07C008D01
:1010C8003A753F0A755905755A00E537C3941150AA
:1010D80005120B998006900587E0F537AE2AAF2BED
:1010E800E5372FFF50010E74641260DD8E2A8F2BB6
:1010F80090007DE0B40146E56775F00A84FF7E0044
:101108008F37E56775F00A84ADF07C008D3A753F3E
:101118000A755905755A6CE537C394115005120BB9
:101128009980069005F3E0F537AE2AAF2BE5372F07
:10113800FF50010E74641260DD8E2A8F2B90008C94
:10114800E0B40249E569C3944175F00584FF7E0067
:101158008F37E56975F00584ADF07C008D3A753FF1
:1011680005755906755A00E537C394135005120BD7
:10117800998006900689E0F537AE2AAF2BE5372F20
:10118800FF50010E74641260DD8E2A8F2B9000CE02
:10119800E0B40202800302124AE55E75F01584FF8E
:1011A8007E008F37E55E75F01584ADF07C008D3AD2
:1011B800753F15755903755AF4E537C3940B5005F7
:1011C800120B998006900475E0F537E53775F0FF46
:1011D800A4FFAEF09000CFE08E048F05FF12608967
:1011E800ED900068F0E56575F078A4FFAEF074FF47
:1011F8008E048F05FF1260898C598D5A74028C06F3
:101208008D071200398F37AC59AD5A7404FF12603C
:10121800B48D3A753F04755906755A28E537C39455
:101228001D5005120B9980069006BBE0F537AE2AD3
:10123800AF2BE5372FFF50010E74641260DD8E2A44
:101248008F2B90007BE0B4025DE56075F064A4FF2D
:10125800AEF074081200398E5B8F5C74058E048FB3
:1012680005FF1260898D37AE5BAF5C74058E048F05
:1012780005FF1260B48D3A753F05755905755ADE3C
:10128800E537C394135005120B998006900667E062
:10129800F537AE2AAF2BE5372FFF50010E746412D5
:1012A80060DD8E2A8F2B9000BDE0703C900044E0FA
:1012B80075F00584FF7E008F37900044E075F005D7
:1012C80084ADF07C008D3A753F05755905755AC097
:1012D800E537C3941D5005120B998006900653E01C
:1012E800F537E537900070F022900084E0B40117DC
:1012F8009007BDE0252BFFAE2A50010E9000D8E0E4
:101308001260DD8E2A8F2B9000FCE0B4011490004F
:10131800FDE0A851B8000495525007E55EC3955FFB
:10132800400280129000A6E0252BFFAE2A50010E45
:101338008E2A8F2B802F900084E0B40316A228B346
:10134800B350109007C0E0C39405A851B8000695A3
:1013580052400280109000A6E0252BFFAE2A5001D3
:101368000E8E2A8F2B90007EE0B4020280030215B5
:101378004D900081E0602FE566D3944640289000A8
:101388000FE0FEA3E0FF9000BCE075F003A4FDAC05
:10139800F0EFD39DEE9C400E9000E0E0A851B8001D
:1013A80005D39552500302154D9000C9E0855EF0B3
:1013B800A4FFAEF0740512609974071200398E59B3
:1013C8008F5A900088E0A851B800049552501290A6
:1013D8000089E075F002A4FDACF0EFC39DEE9C40DF
:1013E8000302154DE55E75F00B84FF7E009006063E
:1013F8001260C0FEE0FFEE900080E0FEEF8E0088F5
:10140800F0A4FFAEF074648E048F05FF1260898C1F
:10141800598D5A900044E075F018A4FFAEF0900082
:10142800C7E08E048F05FF1260898C068D07900631
:101438001E1260C0AE59AF5AE012609974648E04EF
:101448008F05FF1260898C598D5AE564A859B80038
:1014580077D3955A4072E564C3955AFFE49559FECF
:101468008E598F5A7428BE00039F500C755A2875E0
:101478005900740D900045F0AE59AF5A900081E0C4
:1014880012609974288E048F05FF1260898C598D1B
:101498005AAE28AF29740A8E048F05FF1260898D11
:1014A800068C07AC59AD5ACFCECF120003740A8E02
:1014B800048F05FF1260898C598D5AAE28AF291206
:1014C80060E58E288F29807DE564A859B8000495C9
:1014D8005A5072AE59AF5AE5641260DD8E598F5A70
:1014E8007428BE00039F500C755A28755900740D56
:1014F800900045F0AE59AF5A900081E0126099749F
:10150800288E048F05FF1260898C598D5AAE28AF3A
:1015180029740A8E048F05FF1260898D068C07AC2A
:1015280059AD5ACFCECF120003740A8E048F05FF2F
:101538001260898C598D5AAE28AF29EF2DFDEE3CEB
:10154800FC8C288D29229000DCE0B4026AE55E75E7
:10155800F00884FF7E008F37E55E75F00884ADF0F3
:101568007C008D3A753F08755901755AE0E537C317
:10157800943F5005120B998006900275E0F5378567
:10158800372D752C00AE2CAF2DAC2AAD2B120003D5
:1015980074648E048F05FF1260898C2C8D2D900049
:1015A80079E08C068D0712609974648E048F05FFAC
:1015B8001260898C2C8D2DAE28AF29AC2AAD2B1248
:1015C800000374648E048F05FF1260898C288D29AE
:1015D800900079E08C068D0712609974648E048FF0
:1015E80005FF1260898C288D29A20D401DAE51AFD0
:1015F800527405BE00039F5002D20DE560D394CC0F
:101608004008D2017411900045F09000DBE0B4026C
:10161800089000DDE0640160028035AE28AF29E55E
:101628006A12609974E78E048F05FF1260898C280E
:101638008D299000DCE0B40217AE2CAF2DE56A12BC
:10164800609974E78E048F05FF1260898C2C8D2DAC
:1016580090009BE05402601B900092E0A851B800F3
:1016680012D39552400DA20DB3B35007E560C39451
:101678009A40028028AE35AF36900090E075F002AF
:10168800A4FDACF0EF2DFDEE3CFC74022DFD5001E5
:101698000CE560BC0007D39D4003754301856036A7
:1016A800753500E54370030217919000EEE0C3958D
:1016B8004350030217839000FEE0C394025076E57E
:1016C8006675F00A84FF7E009005761260C0E0F52A
:1016D8005A755900AE59AF5A900091E0126099744A
:1016E800648E048F05FF1260898C5B8D5C9000EE20
:1016F800E004C395438C068D071260999000EEE0D4
:101708008E048F05FF1260898C5B8D5CAE28AF2933
:10171800EF2DFDEE3CFC8C288D299000DCE0B40216
:1017280012AE2CAF2DAA5BAB5CEF2BFBEE3AFA8A1C
:101738002C8B2D80469000EEE004C39543854BF03A
:10174800A4FFAEF09000EEE08E048F05FF126089D2
:101758008C5B8D5CAE28AF29EF2DFDEE3CFC8C2810
:101768008D299000DCE0B40212AE2CAF2DAA5BAB41
:101778005CEF2BFBEE3AFA8A2C8B2D05439000EE9A
:10178800E0C39543500375430090009BE05401600B
:101798001B90008FE0A851B80012D39552400DA2BB
:1017A8000DB3B35007E55EC394CC4002802590008A
:1017B8008DE075F003A4FFAEF0E5402FFF50010E59
:1017C80074032FFF50010EE55EBE0007D39F400350
:1017D800754401855E40E54470030218C49000EF2B
:1017E800E0C3954450030218B69000FEE0C394028B
:1017F8005076E56675F00A84FF7E009005761260E3
:10180800C0E0F55A755900AE59AF5A90008EE012F3
:10181800609974648E048F05FF1260898C5B8D5CFF
:101828009000EFE004C395448C068D0712609990F0
:1018380000EFE08E048F05FF1260898C5B8D5CAE33
:1018480028AF29EF2DFDEE3CFC8C288D299000DC7B
:10185800E0B40212AE2CAF2DAA5BAB5CEF2BFBEE13
:101868003AFA8A2C8B2D80469000EFE004C3954409
:10187800854CF0A4FFAEF09000EFE08E048F05FFDA
:101888001260898C5B8D5CAE28AF29EF2DFDEE3C94
:10189800FC8C288D299000DCE0B40212AE2CAF2D10
:1018A800AA5BAB5CEF2BFBEE3AFA8A2C8B2D054436
:1018B8009000EFE0C3954450037544009000F1E0B8
:1018C8002529FFAE2850010E8E288F299000A0E010
:1018D800A828B80004952950099000A0E0F52975BA
:1018E80028009000DCE0B4020D9000A0E0A82CB81D
:1018F8000006952D400280099000A0E0F52D752C7A
:1019080000229000DCE0B401028003021A15A20D47
:10191800B35003021A139000A7E0B40168AE28AFD1
:1019280029AC51AD52120003743C8E048F05FF128E
:1019380060899000B7E0BC00109D400D9000B9E0B0
:10194800A828B8000495295002D202AE28AF29ACC5
:1019580051AD52120003743C8E048F05FF1260894A
:101968009000B7E0C3940ABC0015D39D40119000C5
:10197800B9E0C39405A828B80005D395295002807A
:1019880002C2028068AE28AF29AC51AD52120003E2
:1019980074788E048F05FF1260899000B7E0BC0050
:1019A800109D400D9000B9E0A828B8000495295072
:1019B80004D2028038AE28AF29AC51AD52120003D0
:1019C80074788E048F05FF1260899000B7E0C39485
:1019D8000ABC0015D39D40119000B9E0C39405A836
:1019E80028B80005D3952950028002C202A202B38A
:1019F8004019AE28AF299000B8E012609974648E3F
:101A0800048F05FF1260898C288D298002C202A2EA
:101A180000B34006A201B3B35009900015E4F0A347
:101A2800F08024AE28AF297400D39F74019E400C27
:101A3800900015E528F0A3E529F0800B74FF9000CD
:101A480015F8E4F0E8A3F09000BEE0D39402400C4F
:101A58009000A9E07006A20DB3B34002801AAE2828
:101A6800AF2974021260998E288F29AE2CAF2D747D
:101A7800021260998E2C8F2D9000A7E0B4011AAE47
:101A880028AF2974021260998E288F29AE2CAF2DA9
:101A980074021260998E2C8F2DAE28AF29745E12B5
:101AA8006099740A8E048F05FF1260898C288D292D
:101AB8009000DCE0B40217AE2CAF2D745E12609972
:101AC800740A8E048F05FF1260898C2C8D2DAE2828
:101AD800AF297402BE000AD39F40067529027528F3
:101AE80000AE2CAF2D7402BE000AD39F4006752DA0
:101AF80002752C00900013E528F0A3E529F0229048
:101B08000044E09003761260CBE0F54175426490A2
:101B18000044E0FE9000B2E0D39E4037E55E75F0E9
:101B28000884FF7E008F37E55E75F00884ADF07C91
:101B3800008D3A753F08755903755A96E537C39471
:101B48001F5005120B99800690042BE0F537853756
:101B5800428035E55E75F00884FF7E008F37E55ECC
:101B680075F00884ADF07C008D3A753F087559030F
:101B7800755AB6E537C3941F5005120B9980069025
:101B8800044BE0F537853742229000E8E0F53C75D4
:101B98003F11755904755A00AE51AF52E53C75F0C6
:101BA8000FA4FDACF0EDD39FEC9E4021E53C8E04E4
:101BB8008F05FF126089ED75F010A4FFAEF0E55EA9
:101BC80075F01184FD7C00ED2FF53D800EE55E7506
:101BD800F01184FF7E00EF24F0F53D853D37E55E8A
:101BE80075F01184AFF07E008F3A120B9985373E5D
:101BF800AE51AF529000E8E075F00FA4FDACF0EDE7
:101C0800D39FEC9E4028755904755A10853D3712AC
:101C18000B99853E38853739AE51AF52E53C8E0475
:101C28008F05FF1260B48D3A853C3B120C13853743
:101C380041754264229000E8E0F53C753F11755902
:101C480004755A00AE51AF52E53C75F00FA4FDACD7
:101C5800F0EDD39FEC9E4021E53C8E048F05FF12EA
:101C68006089ED75F010A4FFAEF0E56075F01184A1
:101C7800FD7C00ED2FF53D800EE56075F01184FFC9
:101C88007E00EF24F0F53D853D37E56075F0118461
:101C9800AFF07E008F3A120B9985373EAE51AF52A6
:101CA8009000E8E075F00FA4FDACF0EDD39FEC9E3A
:101CB8004028755904755A10853D37120B99853E91
:101CC80038853739AE51AF52E53C8E048F05FF1287
:101CD80060B48D3A853C3B120C13853741754264DC
:101CE8009000E3E0B40479900044E0FE9000B2E094
:101CF800D39E4037E55E75F00884FF7E008F37E598
:101D08005E75F00884ADF07C008D3A753F08755912
:101D180003755A96E537C3941F5005120B99800630
:101D280090042BE0F5378537428035E55E75F0087D
:101D380084FF7E008F37E55E75F00884ADF07C0087
:101D48008D3A753F08755903755AB6E537C3941F20
:101D58005005120B99800690044BE0F53785374201
:101D68002290007CE0B4013BE56675F00A84FF7EB2
:101D7800008F37E56675F00A84ADF07C008D3A7502
:101D88003F0A755905755A12E537C3941150051263
:101D98000B998006900599E0F537E5422537C394FD
:101DA80064F54290007DE0B4013BE56775F00A8474
:101DB800FF7E008F37E56775F00A84ADF07C008DF3
:101DC8003A753F0A755905755A7EE537C39411501F
:101DD80005120B998006900605E0F537E542253790
:101DE800C39464F542E5412542F534900084E0B49B
:101DF80002109007BCE02534FE9000D8E0F4042ED1
:101E0800F5349000DBE0D394014040E56AC394E7E1
:101E1800501D74E7C3956AFE9007BEE08E00F5F08A
:101E2800E884FF7E008F37E5342537F534801CE5DC
:101E38006AC394E7FE9007BEE08E00F5F0E884FFE1
:101E48007E008F37E534C39537F534A20D4006E59B
:101E5800412464F534E534D394644009E534C394EB
:101E680064F53480037534009000B4E0C3953450B1
:101E7800069000B4E0F53422D20090006EE0A8513C
:101E8800B800049552504190006EE0A851B8000483
:101E98009552500375340F90006EE004A851B800B5
:101EA800049552500375340A90006EE02402A8513C
:101EB800B8000495525005753405C20090006EE0D4
:101EC80060067409900045F0C2387E017F009000DA
:101ED800BAE01260999000C9E08E048F05FF126085
:101EE80089E55EBC0017D39D40139000C3E0B4029F
:101EF80004D2388002C200740A900045F09000BBFA
:101F0800E0C3956650159000CDE0A851B80004953F
:101F1800525002C200740B900045F0E566C3946409
:101F2800501D900113E0600D900113E0A851B80016
:101F380006955240028008C200740B900045F0A23A
:101F48000040037534059000FCE0B401149000FDD6
:101F5800E0A851B8000495525007E55EC3955F406C
:101F68000280089000A5E0F534803A900084E0B43F
:101F78000306A228B3B34002802B9007C0E0C394A5
:101F880005A851B800049552500C9000A5E0F5340E
:101F9800740C900045F09007C0E0A851B800049573
:101FA800525002C20085346B900076E02534FE90D2
:101FB8000044E075F01E84FC7F00EE2CF53422907E
:101FC8000044E075F00584FF7E008F37900044E000
:101FD80075F00584ADF07C008D3A753F05755903A1
:101FE800755AD69000C7E01475F00584FF7E00E5A9
:101FF80037BE00039F5005120B99800BE5379004FC
:102008004C1260CBE0F537E5379007BFF09007BF7B
:10201800E0FE9000B6E0C39E50089000B6E090073E
:10202800BFF022E56675F00A84FF7E0090057612FF
:1020380060C0E0F546E546D394644010E546C39495
:102048006475F00F84FF7E008F468003754600900C
:102058000099E02546F546229007B0E0FEA3E0FF90
:102068007404120039E55E126099740F8E048F05AE
:10207800FF1260899007AEECF0A3EDF090008CE0C1
:10208800B40262E569C3944175F00584FF7E008F50
:1020980037E56975F00584ADF07C008D3A753F052C
:1020A800755906755A14E537C394175005120B99DC
:1020B800800690069DE0F5379007AEE0FEA3E0FFAE
:1020C800740A8E048F05FF126089E5378C068D0728
:1020D800126099740A8E048F05FF1260899007AE0A
:1020E800ECF0A3EDF09007AEE0FEA3E0FF9007B49C
:1020F800E0FCA3E0FDEDD39FEC9E400F9007B4E019
:10210800F8A3E09007AEC8F0A3C8F0229006BDE09F
:10211800903419F8282873804C85527280479000B3
:10212800C9E0855EF0A4FFAEF074081200398F7222
:102138008033856072802E856672802985677280FB
:1021480024856872801F856972801A856A72801575
:102158008565728010856472800B856B728006902D
:052168000016E0F57215
:1034190002211F02212102212602213A02213F0213
:10342900214402214902214E02215302215802213D
:073439005D02216202216720
:10216D009006BEE0FE9006BFE0D39E404B9006BDAC
:10217D00E0B404189006BFE0C395725002D22990C6
:10218D0006BEE0D395724002C229802A9006BEE0B9
:10219D00C3957250099006BFE0D39572500280022C
:1021AD00D2299006BEE0D3957250099006BFE0C3C8
:1021BD0095725002C229802A9006BEE0D3957240D6
:1021CD00099006BFE0C3957240028002C2299006B5
:1021DD00BEE0C3957240099006BFE0D395724002F0
:1021ED00D229229006C1E0903440F8282873804C03
:1021FD0085527280479000C9E0855EF0A4FFAEF075
:10220D0074081200398F728033856072802E856656
:10221D007280298567728024856872801F85697236
:10222D00801A856A7280158565728010856472804A
:0C223D000B856B728006900016E0F572B5
:103440000221FB0221FD02220202221602221B029D
:10345000222002222502222A02222F0222340222C4
:073460003902223E02224363
:102249009006C2E0FE9006C3E0D39E405F9006C1AF
:10225900E0B404189006C3E0C395725002D22A90E4
:1022690006C2E0D395724002C22A803E9006C2E0BF
:10227900C3957250099006C3E0D39572500280024B
:10228900D22A9006C2E0D3957250099006C3E0C3E2
:1022990095725002C22A9006C1E0B401099000D596
:1022A900E0D3956050028002C22A802A9006C2E0DB
:1022B900D3957240099006C3E0C39572400280022B
:1022C900C22A9006C2E0C3957240099006C3E0D3C2
:1022D90095724002D22A229006C5E0903467F82808
:1022E9002873804C85527280479000C9E0855EF062
:1022F900A4FFAEF074081200398F728033856072C2
:10230900802E85667280298567728024856872802F
:102319001F856972801A856A7280158565728010B9
:10232900856472800B856B728006900016E0F572E9
:103467000222EB0222ED0222F202230602230B02C2
:10347700231002231502231A02231F0223240223E7
:073487002902232E0223336A
:102339009006C6E0FE9006C7E0D39E404B9006C5C6
:10234900E0B404189006C7E0C395725002D22B90EE
:1023590006C6E0D395724002C22B802A9006C6E0D9
:10236900C3957250099006C7E0D395725002800256
:10237900D22B9006C6E0D3957250099006C7E0C3E8
:1023890095725002C22B802A9006C6E0D3957240FE
:10239900099006C7E0C3957240028002C22B9006DD
:1023A900C6E0C3957240099006C7E0D39572400212
:1023B900D22B229006C9E090348EF8282873804CDD
:1023C90085527280479000C9E0855EF0A4FFAEF0A7
:1023D90074081200398F728033856072802E856689
:1023E9007280298567728024856872801F85697269
:1023F900801A856A7280158565728010856472807D
:0C2409000B856B728006900016E0F572E7
:10348E000223C70223C90223CE0223E20223E7024C
:10349E0023EC0223F10223F60223FB022400022472
:0734AE000502240A02240FAD
:102415009006CAE0FE9006CBE0D39E404B9006C9DD
:10242500E0B404189006CBE0C395725002D22C900C
:1024350006CAE0D395724002C22C802A9006CAE0F3
:10244500C3957250099006CBE0D395725002800275
:10245500D22C9006CAE0D3957250099006CBE0C302
:1024650095725002C22C802A9006CAE0D39572401C
:10247500099006CBE0C3957240028002C22C9006FB
:10248500CAE0C3957240099006CBE0D3957240022D
:10249500D22C229006CDE09034B5F8282873804CD4
:1024A50085527280479000C9E0855EF0A4FFAEF0CA
:1024B50074081200398F728033856072802E8566AC
:1024C5007280298567728024856872801F8569728C
:1024D500801A856A728015856572801085647280A0
:0C24E5000B856B728006900016E0F5720B
:1034B5000224A30224A50224AA0224BE0224C302D4
:1034C50024C80224CD0224D20224D70224DC0224FB
:0734D500E10224E60224EBF2
:1024F1009006CEE0FE9006CFE0D39E404B9006CDF5
:10250100E0B404189006CFE0C395725002D22D902A
:1025110006CEE0D395724002C22D802A9006CEE00D
:10252100C3957250099006CFE0D395725002800294
:10253100D22D9006CEE0D3957250099006CFE0C31C
:1025410095725002C22D802A9006CEE0D39572403A
:10255100099006CFE0C3957240028002C22D900619
:10256100CEE0C3957240099006CFE0D39572400248
:10257100D22D229006D1E09034DCF8282873804CCB
:1025810085527280479000C9E0855EF0A4FFAEF0ED
:1025910074081200398F728033856072802E8566CF
:1025A1007280298567728024856872801F856972AF
:1025B100801A856A728015856572801085647280C3
:0C25C1000B856B728006900016E0F5722E
:1034DC0002257F02258102258602259A02259F025C
:1034EC0025A40225A90225AE0225B30225B8022582
:0734FC00BD0225C20225C735
:1025CD009006D2E0FE9006D3E0D39E404B9006D10C
:1025DD00E0B404189006D3E0C395725002D22E9049
:1025ED0006D2E0D395724002C22E802A9006D2E028
:1025FD00C3957250099006D3E0D3957250028002B4
:10260D00D22E9006D2E0D3957250099006D3E0C336
:10261D0095725002C22E802A9006D2E0D395724058
:10262D00099006D3E0C3957240028002C22E900637
:10263D00D2E0C3957240099006D3E0D39572400263
:10264D00D22E229006D5E0903503F8282873804CC1
:10265D0085527280479000C9E0855EF0A4FFAEF010
:10266D0074081200398F728033856072802E8566F2
:10267D007280298567728024856872801F856972D2
:10268D00801A856A728015856572801085647280E6
:0C269D000B856B728006900016E0F57251
:1035030002265B02265D02266202267602267B02E3
:10351300268002268502268A02268F022694022608
:073523009902269E0226A377
:1026A9009006D6E0FE9006D7E0D39E404B9006D523
:1026B900E0B404189006D7E0C395725002D22F9067
:1026C90006D6E0D395724002C22F802A9006D6E042
:1026D900C3957250099006D7E0D3957250028002D3
:1026E900D22F9006D6E0D3957250099006D7E0C351
:1026F90095725002C22F802A9006D6E0D395724077
:10270900099006D7E0C3957240028002C22F900655
:10271900D6E0C3957240099006D7E0D3957240027E
:10272900D22F229006D9E090352AF8282873804CB8
:1027390085527280479000C9E0855EF0A4FFAEF033
:1027490074081200398F728033856072802E856615
:102759007280298567728024856872801F856972F5
:10276900801A856A72801585657280108564728009
:0C2779000B856B728006900016E0F57274
:10352A0002273702273902273E022752022757026B
:10353A00275C02276102276602276B02277002278F
:07354A007502277A02277FBA
:102785009006DAE0FE9006DBE0D39E404B9006D93A
:10279500E0B404189006DBE0C395725002D2309085
:1027A50006DAE0D395724002C230802A9006DAE05C
:1027B500C3957250099006DBE0D3957250028002F2
:1027C500D2309006DAE0D3957250099006DBE0C36B
:1027D50095725002C230802A9006DAE0D395724095
:1027E500099006DBE0C3957240028002C230900674
:1027F500DAE0C3957240099006DBE0D3957240029A
:10280500D230229006DDE0903551F8282873804CAF
:1028150085527280479000C9E0855EF0A4FFAEF056
:1028250074081200398F728033856072802E856638
:102835007280298567728024856872801F85697218
:10284500801A856A7280158565728010856472802C
:0C2855000B856B728006900016E0F57297
:1035510002281302281502281A02282E02283302F3
:10356100283802283D02284202284702284C022816
:073571005102285602285BFD
:102861009006DEE0FE9006DFE0D39E404B9006DD51
:10287100E0B404189006DFE0C395725002D23190A3
:1028810006DEE0D395724002C231802A9006DEE076
:10289100C3957250099006DFE0D395725002800211
:1028A100D2319006DEE0D3957250099006DFE0C385
:1028B10095725002C231802A9006DEE0D3957240B3
:1028C100099006DFE0C3957240028002C231900692
:1028D100DEE0C3957240099006DFE0D395724002B5
:1028E100D231229006E1E0903578F8282873804CA7
:1028F10085527280479000C9E0855EF0A4FFAEF07A
:1029010074081200398F728033856072802E85665B
:102911007280298567728024856872801F8569723B
:10292100801A856A7280158565728010856472804F
:0C2931000B856B728006900016E0F572BA
:103578000228EF0228F10228F602290A02290F027E
:10358800291402291902291E02292302292802299D
:073598002D02293202293740
:10293D009006E2E0FE9006E3E0D39E404B9006E168
:10294D00E0B404189006E3E0C395725002D23290C1
:10295D0006E2E0D395724002C232802A9006E2E090
:10296D00C3957250099006E3E0D395725002800230
:10297D00D2329006E2E0D3957250099006E3E0C39F
:10298D0095725002C232802A9006E2E0D3957240D1
:10299D00099006E3E0C3957240028002C2329006B0
:1029AD00E2E0C3957240099006E3E0D395724002D0
:1029BD00D23222AE2EAF2F74F5D39F74019E4008F4
:1029CD00782E1260ED022ADA752F01752E00AE51A8
:1029DD00AF52E546BE000DD39F40099000ABE0D34A
:1029ED00954740028023754700E546C39552F57221
:1029FD009000AEE0D395454008E5452572F545803C
:102A0D00069000AEE0F54580020547900087E0D3C3
:102A1D009560401CE55EC3955F4015AE51AF52E524
:102A2D0046BE00039F50099000ACE0D3954840028C
:102A3D00806E9007C3E0A851B800049552500375FD
:102A4D004A009007C3E0A851B8000BD39552400639
:102A5D00E5529007C3F0E54A7041E552C39546F53E
:102A6D0072E572D3940540037572059000ADE0C315
:102A7D0095455007E572C3954540028009E545C36C
:102A8D009572F54580069000ADE0F5459000ADE0FE
:102A9D00D3954540069000ADE0F5457548008002A0
:102AAD000548E54A7016900087E0C39560500DE526
:102ABD00462405A851B8000695524002800F90009B
:102ACD009AE0F545754A0174789007C3F022AE2E51
:102ADD00AF2F74E9D39F74039E4008782E1260EDDA
:102AED00022C79752F01752E00754532A233402ABF
:102AFD0075451990009AE075F002A4FFAEF0E54718
:102B0D00BE0006D39F4002D2330547754A03747841
:102B1D009007C3F0754900022C68AE51AF52E546DF
:102B2D006F4E7003022C68E546BE000DD39F400921
:102B3D009000ABE0D395474002800F754700E54A02
:102B4D00C394035003754519800DE546C39552F5A1
:102B5D0072E5472572F547900087E0D39560400EEA
:102B6D009007C3E0A851B80007D395524002800CDE
:102B7D00054990009AE0B54903754A00E54AB4034A
:102B8D0006A20DB3B34002800A0549E549B43C03E2
:102B9D00754A02E54AB402299007C3E0A851B8006E
:102BAD000ED395524009E5529007C3F07549009038
:102BBD000087E0C39560500975490074789007C38C
:102BCD00F0E54A705A900087E0D39560401CE55EB1
:102BDD00C3955F4015AE51AF52E546BE00039F5001
:102BED00099000ACE0D39548400280087548007507
:102BFD00454B8028E552C39546F572E572D3940591
:102C0D004003757205900087E0D395604008E54854
:102C1D002572F5488006E5482406F548754900E516
:102C2D004A7016900087E0C39560500DE546240567
:102C3D00A851B80006955240028003754A01E54A35
:102C4D00B40118754519054990009AE0B549067506
:102C5D004A0275490074789007C3F0E54575F00A8E
:102C6D00A4FFAEF09007B8EEF0A3EFF022E56E9062
:102C7D00359FF828287390007FE07003022E28906E
:102C8D0000B5E0B401028003022D78900042E0B55A
:102C9D005D028003022D757E017F00E5BE126099F5
:102CAD00E5BD2FFF50010E8E598F5A741012609989
:102CBD0090006DE08E048F05FF1260899007C4ECC3
:102CCD00F0A3EDF0E56A60089000DBE064026002BD
:102CDD0080269000DDE0B4011F9007C4E0FEA3E064
:102CED00FF74E7126099E56A8E048F05FF12608903
:102CFD009007C4ECF0A3EDF090007FE0B4022790B4
:102D0D0007C6E0FEA3E0FF9007C4E0FCA3E0FDEFE3
:102D1D002DFDEE3CFC74018C068D071200399007D9
:102D2D00C4EEF0A3EFF09007C4E0FEA3E0FF900720
:102D3D00C6E0FCA3E0FDEDD39FEC9E4004D23680AF
:102D4D0002B2369007C4E0F8A3E09007C6C8F0A31E
:102D5D00C8F09000B1E064016006A236B3B3400242
:102D6D0080069007C5E0F55E022E26D2367E017FE5
:102D7D0000E5BE126099E5BD2FFF50010E8E598FF3
:102D8D005A741012609990006DE08E048F05FF1239
:102D9D0060899007C4ECF0A3EDF0E56A600890003F
:102DAD00DBE06402600280269000DDE0B4011F903C
:102DBD0007C4E0FEA3E0FF74E7126099E56A8E0494
:102DCD008F05FF1260899007C4ECF0A3EDF0900021
:102DDD007FE0B402279007C6E0FEA3E0FF9007C492
:102DED00E0FCA3E0FDEF2DFDEE3CFC74018C068DA7
:102DFD00071200399007C4EEF0A3EFF09007C4E07E
:102E0D00F8A3E09007C6C8F0A3C8F09000B1E06445
:102E1D000160069007C5E0F55E8003755E009000C9
:102E2D007BE07006756E01022C7A75BB180233F3C8
:102E3D0090007BE07003022FC97E017F00E5BE127A
:102E4D006099E5BD2FFF50010E8E598F5A9000C12C
:102E5D00E0B4010F7E0F7FFFAC59AD5A1260E58EC5
:102E6D00598F5A9000E6E0B40245AE59AF5A900022
:102E7D001FE0FCA3E0FDEDD39FEC9E400A90001FE8
:102E8D00E559F0A3E55AF0AE59AF5A900021E0FC98
:102E9D00A3E0FDEFD39DEE9C400A900021E559F093
:102EAD00A3E55AF0AE59AF5A74041200398F6090F1
:102EBD0000E6E0704CAE59AF5A90001FE0FCA3E065
:102ECD00FDEFD39DEE9C40091260E58E598F5A801F
:102EDD0006755A00755900AE59AF5A7410126099A3
:102EED0090006AE08E048F05FF1260898C598D5A0F
:102EFD0074FFBC0009D39D4005855A608003756041
:102F0D00FE9000B1E0B401028003022FC7A20DB301
:102F1D00B3500E900085E0A851B80005D3955250DE
:102F2D0003022FBC900086E075F019A4FFAEF0905F
:102F3D0000C9E08E048F05FF1260899000C2E08504
:102F4D0060F0A4FFAEF074648D028C038E048F05C7
:102F5D00FF126089EA2DFDEB3CFC8C598D5AE56A18
:102F6D00600F9000DBE0B402089000DDE0640160CA
:102F7D00028017AE59AF5A74E7126099E56A8E0454
:102F8D008F05FF1260898C598D5AAE59AF5A900733
:102F9D00C4E0FCA3E0FDEDD39FEC9E4005855A5E99
:102FAD00800BA236B340069007C5E0F55E800BA2FC
:102FBD0036B340069007C5E0F55E8003756000905E
:102FCD00007EE07006756E02022C7A75BB19023315
:102FDD00F390007EE0700302307EE55DD3955040A6
:102FED000302307C90001DE0FEA3E0FFE56412605B
:102FFD00DD90001DEEF0A3EFF07E017F00E5BE1227
:10300D006099E5BD2FFF50010E8E598F5A9000EB40
:10301D00E07013740A12609974518E048F05FF12BB
:10302D0060898D648019AE59AF5A740A1260998FF8
:10303D00048E057E017F95CDCCCD125F878F64E523
:10304D0064D39464400375646490001DE0FEA3E0B6
:10305D00FFE5642FFF50010E90001DEEF0A3EFF081
:10306D00900082E0048E048F05FF1260898D6480CC
:10307D00037564329000CEE07006756E03022C7AF3
:10308D0075BB130233F39000CEE0604A7E017F00E2
:10309D00E5BE126099E5BD2FFF50010E8E598F5A76
:1030AD0074041200398F659000D0E08565F0A4FDA1
:1030BD00ACF07464FF1260898D659000CFE085657A
:1030CD00F0A4FFAEF074FF8E048F05FF126089ED42
:1030DD00900069F0800375650090007CE0700675C6
:1030ED006E04022C7A75BB170233F390007CE0B4AA
:1030FD000102800302318C7E017F00E5BE126099D2
:10310D00E5BD2FFF50010E8E598F5A9007C8E06014
:10311D00199007C8E014905A0512008CE493FC74C2
:10312D000193FDEDC39FEC9E400280069007C8E021
:10313D0014F09007C8E0C394B3501DAE59AF5A9028
:10314D0007C8E004905A0512008CE493FC740193B7
:10315D00FDEFC39DEE9C400280069007C8E004F091
:10316D009007C8E0FE9000A2E08E0088F0A4FFAEAC
:10317D00F074648E048F05FF1260898D668003756F
:10318D00660090007DE07006756E05022C7A75BBA9
:10319D00160233F390007DE0B40102800302323554
:1031AD007E017F00E5BE126099E5BD2FFF50010E37
:1031BD008E598F5A9007C9E060199007C9E0149095
:1031CD005B6F12008CE493FC740193FDEDC39FECD7
:1031DD009E400280069007C9E014F09007C9E0C335
:1031ED0094B3501DAE59AF5A9007C9E004905B6F70
:1031FD0012008CE493FC740193FDEFC39DEE9C4093
:10320D000280069007C9E004F09007C9E0FE900027
:10321D00A8E08E0088F0A4FFAEF074648E048F05D4
:10322D00FF1260898D67800375670075BB1F0233C0
:10323D00F37E017F00E5BE126099E5BD2FFF5001C1
:10324D000E8E598F5A740912609974E68E048F058B
:10325D00FF1260898D69900084E07006756E07021B
:10326D002C7A75BB150233F3900084E070030233A2
:10327D008F7E017F00E5BE126099E5BD2FFF5001E5
:10328D000E8E598F5A74041200398F68900084E0A5
:10329D00B401159000D8E08568F0A4FFAEF0740776
:1032AD00120039EF9007BDF0900084E0B402159044
:1032BD0000D8E08568F0A4FFAEF07407120039EF76
:1032CD009007BCF0900084E0B40302800302338DBC
:1032DD009000C5E070389000D8E0601CE568C3949C
:1032ED00195002D228E568D394644002C228900098
:1032FD00A4E09007C0F08014E568C394195002D281
:10330D0037E568D394324002C237C22880639000FB
:10331D00A4E070349000D8E08568F0A4FFAEF0749E
:10332D00FF8E048F05FF126089ED9007C0F0AE513E
:10333D00AF52741EBE0006D39F4002D228E560D363
:10334D0094E54002C2288029E568C3940A500DAE69
:10335D0051AF52741EBE0004D39F50028002D2287A
:10336D00E560D394E54002C2289000A4E09007C028
:10337D00F09007C0E0C39405500674059007C0F0A7
:10338D0080037568009000DBE07006756E08022CF6
:10339D007A75BB1480509000DBE060397E017F00B0
:1033AD00E5BE126099E5BD2FFF50010E8E598F5A63
:1033BD00EFD39421EE940E4005756AFF8015AE593A
:1033CD00AF5A741012609974E38E048F05FF12606A
:1033DD00898D6A8003756A0090007FE0600575BB7A
:0633ED001A800375BB18F5
:10359F00022C83022E3D022FDE0230930230F802FE
:0B35AF0031A102323E0232750233A34C
:0533F300056ED2EC2282
:0960CB002582F5825002058322B2
:0F008C0025E050020583258250020583F582226C
:10606800EF2F500205832582F582E5833E2EF583C6
:016078002205
:1060DD00CFC39FFF50011E22C3EF9DFFEE9CFE22FA
:0860ED000806B60002180622A5
:0D60A700A3E004F07006120049E004F022AE
:0E003900048007C3CE13CECF13CFD5E0F6223E
:105F8700BC000FBE0008ED8FF084FFADF022E4FEE9
:105F9700FF22BE000DEF60FE54F0606F20E70302A2
:105FA700603DEAC0E0EBC0E078017A0075F001EEF1
:105FB70020E710EF25E0FFEE33FE0AC5F023C5F01A
:105FC70030E7F0EA5407F9096A7A007B00600108B4
:105FD700C3EC9E40167004ED9F4010ED9FFDEC9EB4
:105FE700FCE5F0CA4ACA03F5F08005E5F003F5F0D1
:105FF700C3EE13FEEF13FFD9D77908CACBCAD8D09F
:10600700EAFEEBFFD0E0FBD0E0FA22EC8FF084FC55
:10601700ED54F045F0C48FF084FEEDC454F045F024
:10602700C48FF084FDEEC4FE54F02DFFEE540F3CF8
:10603700FEADF07C0022790078008FF0EC7E08201E
:10604700E70DC3CD33CD33C933C9C833C8DEF084B8
:1060570049F9E5F08FF0BE00E6FD7C00E9FFE8FEB8
:016067002216
:0E609900F88FF0A4FFE5F0CE88F0A42EFE22D2
:10000300EF8DF0A4F9A8F0EF8CF0A428F8EE8DF0B2
:06001300A428FEE9FF2213
:10607900600D782B026083007830D8FED5E0F822D5
:10608900EEC0E07E00125F87EFFDEEFCD0E0FE225D
:0C60B400EEC0E07E00125F87D0E0FE220C
:03001B0002001EC2
:0300530002005652
:03009B00020071EF
:030000000260D4C7
:0960D40075817475D000023DEEE7
:0B60C000E5822FF582E5833EF5832288
:0A0049000582D5820215831582227C
:10001E00C0E0C0F0C083C082C0D075D000123D28B1
:0B002E00D0D0D082D083D0F0D0E032E0
:10005600C0E0C0F0C083C082C0D075D000123D2B76
:10006600D0D0D082D083D0F0D0E032C0E0C0F0C093
:1000760083C082C0D075D000123DB0D0D0D082D01F
:0600860083D0F0D0E0324F
:00000001FF
